:1000000000000000000000008316403081007F30B7
:100010008600831221308400F9308000840AF83091
:100020008000840AF8308000840AF7308000840A57
:10003000F7308000840AF6308000840AF6308000B1
:10004000840AF5308000840AF5308000840AF43098
:100050008000840AF4308000840AF4308000840A2E
:10006000F3308000840AF3308000840AF33080008B
:10007000840AF3308000840AF3308000840AF3306D
:100080008000840AF3308000840AF3308000840A00
:10009000F3308000840AF4308000840AF430800059
:1000A000840AF4308000840AF5308000840AF53038
:1000B0008000840AF6308000840AF6308000840ACA
:1000C000F7308000840AF7308000840AF83080001E
:1000D000840AF8308000840AF9308000840AFA30FB
:1000E0008000840AFA308000840AFB308000840A91
:1000F000FB308000840AFC308000840AFC308000E1
:10010000840AFD308000840AFD308000840AFE30BD
:100110008000840AFE308000840AFE308000840A59
:10012000FF308000840AFF308000840AFF308000A6
:10013000840AFF308000840AFF308000840AFF3088
:100140008000840AFF308000840AFF308000840A27
:10015000FF308000840AFE308000840AFE30800078
:10016000840AFE308000840AFD308000840AFD305D
:100170008000840AFC308000840AFC308000840AFD
:10018000FB308000840AFB308000840AFA30800053
:10019000840AFA308000E10A0319E20A8B1CE52880
:1001A0008B1000006108E3006208E400E101E20155
:1001B000E501E601E701E30DE40DE30DE40DFC309C
:1001C000E305213084008617CB28621ACE28670801
:1001D0006202031CFC2866086102031C00296308F4
:1001E000E50764080318640AE6070318E70A840AA7
:1001F0000008E8008617CE2800000000000000007C
:10020000000000000000841A0413E80A6808860051
:08021000CB2802010403FA3FB0
:00000001FF
